:10000000BEEF22F000000000000000000000000031
:1000100000000000000000000000000000000000E0
:1000200000000000000000000000000000000000D0
:10003000000000000000000000000000000022118D
:100040000000000000000000571300000000000046
:1000500000000000000000000000000000000000A0
:100060000000000000000000000000000000000090
:100070000000000000000000000000000000000080
:100080000000000000000000000000000000000070
:100090000000000000000000000000000000000060
:0C00A00000000000000000000000000054
:0C00AC00000E3D01F9BF010E006E1200B5
:0C00B800000E3D01E1BF010E006E1200C1
:0400C400F9DF12004E
:0400C800F1DF120052
:0800CC000AAE029E000E1200B4
:1000D400F9DF005202E10000FBD76000F7F7EAFD08
:0200E400120008
:1000E600EEDF005202E10000FBD76000F7F7D2FD19
:0200F6001200F6
:1000F8000B820BAE86EF00F00368026801680068A7
:080108000A360232FF0E12005C
:100110000B840BAE93EF00F0010E036E026A016ACE
:0A012000006A0A360232FF0E1200D8
:0E012A00026A016A006A086A036A000E120087
:100138000CB0DEEF00F00CA284EF01F00E6A000EA6
:100148000264F5EF00F0F00E0214D8A4C0EF00F03E
:10015800023A01380F0B02260138F00B016E003805
:100168000F0B01260038F00B006E08380F0B002625
:100178000838F00B086E0E84D89002BED9EF00F054
:1001880008360036013602360E2A02BED9EF00F0D4
:1001980008360036013602360E2A02BED9EF00F0C4
:1001A80008360036013602360E2A0E5003647AEFFE
:1001B80001F0035E0BBC08AE7FEF01F0D880800E23
:1001C80008640030000E002201220222D8A07FEF2E
:1001D80001F0023201320032034A84EF01F07FEF6E
:1001E80001F001C002F000C001F008C000F0086A88
:1001F800000E0E8602642CEF01F0F00E0214D8A453
:1002080014EF01F0023A01380F0B02260138F00B07
:10021800016E00380F0B01260038F00B006E0E84BB
:10022800D89002BED9EF00F00036013602360E2A09
:1002380002BED9EF00F00036013602360E2A02BEA1
:10024800D9EF00F00036013602360E2AD9EF00F059
:1002580001C002F000C001F0006A000E0E960E8880
:10026800026459EF01F0F00E0214D8A444EF01F033
:10027800023A01380F0B02260138F00B016E0E848A
:10028800D89002BED9EF00F0013602360E2A02BE1F
:10029800D9EF00F0013602360E2A02BED9EF00F07F
:1002A800013602360E2AD9EF00F001C002F0016AC9
:1002B800000E0E86026489EF01F0F00E0214D8A435
:1002C80068EF01F0023A0E84D89002BED9EF00F030
:1002D80002360E2A02BED9EF00F002360E2A02BEFE
:1002E800D9EF00F002360E2AD9EF00F0010E0C6E9D
:1002F8000BDF8CEF01F0020E0C6EE4DE8CEF01F0E8
:10030800040E0C6EF5DE8CEF01F0080E0C6E09DFA2
:020318001200D1
:08031A00FCC1FDF1DADE120066
:08032200FCC1FDF1DFDE120059
:08032A00FCC1FDF1DBDE120055
:08033200FCC1FDF1CEDE12005A
:10033A000D6A086A0050D8B4000C04180A6E0ABE86
:10034A000D1E0B6A04AE02D0041E042A00AE02D0AF
:10035A00001E002A005004100A6E0ABE1FD0045064
:10036A00085E003600340836045008260036060EA9
:10037A000C6E00340836045000B0085E00A008264F
:10038A0000360C2EF6D700A008260BB015D00DAEFD
:10039A00000C001E002A081E082A000C04AE09D010
:1003AA0000BE04D00050086E006AF1D7006A002A25
:1003BA00000C001E0B2AD3D7082A0450085CD8A4C4
:0E03CA00E6D7086A002A00AEE2D7FF0C120048
:1003D800086A080E0C6E003408360450085ED8B05F
:0E03E80002D00826D89000360C2EF5D7120051
:1003F6000134083609360450085E0550D8A0053C7D
:10040600095E003601360F0E0C6E013408360936C9
:10041600045000A006D0085E0550D8A0053C095E31
:1004260005D008260550D8B0053C09260036013609
:100436000C2EEBD700B006D0045008260550D8B0D5
:08044600053C0926000012002C
:10044E00D250026ED29E0500FF6A0150FE6E005021
:08045E00FD6E02BED28E1200F9
:10046600025006180E6E086A096A0B6A0350076482
:1004760026EF03F006500A6E068E028E03500B6EB0
:100486000750036E000E0B6476EF02F00B50075E0A
:10049600D8B417EF03F0070E0764E5EF02F0075E26
:1004A60000C008F001C000F002C001F0026A074E69
:1004B60017EF03F00764BAEF02F0075E00C008F01A
:1004C60001C000F0016A074E17EF03F0076498EFCA
:1004D60002F0075E00C008F0006A074E17EF03F04F
:1004E60007647FEF02F00AC002F005C001F004C005
:1004F60000F0086A40EF04F0030E07648AEF02F08A
:10050600075E08380F0B086E074E17EF03F0D890FA
:100516000832074E17EF03F0D8900832074E17EF50
:1005260003F0D890083217EF03F0030E0764A9EF23
:1005360002F0075E08380F0B086E0038F00B08262D
:1005460000380F0B006E074E17EF03F0D8900032FD
:100556000832074E17EF03F0D89000320832074EE4
:1005660017EF03F0D8900032083217EF03F0030EAE
:100576000764D1EF02F0075E08380F0B086E0038EB
:10058600F00B082600380F0B006E0138F00B002622
:1005960001380F0B016E074E17EF03F0D8900132AA
:1005A60000320832074E17EF03F0D89001320032BE
:1005B6000832074E17EF03F0D890013200320832A6
:1005C60017EF03F0030E076402EF03F0075E083827
:1005D6000F0B086E0038F00B082600380F0B006E64
:1005E6000138F00B002601380F0B016E0238F00BB4
:1005F600012602380F0B026E074E17EF03F0D89054
:100606000232013200320832074E17EF03F0D8905B
:100616000232013200320832074E17EF03F0D8904B
:100626000232013200320832096A000E0EAE0BEFBA
:1006360004F0081E001E011E021E082A00220122C6
:1006460002220BEF04F00750D8A42CEF03F040EF82
:1006560004F0096A02C00AF0028E068E0750035C97
:10066600076ED8B4FEEF03F0070E0764CCEF03F075
:10067600075E0450096E0550046E0650056E066A44
:10068600074EFEEF03F0070E0764A1EF03F0075EC7
:100696000450096E0550046E056A074EFEEF03F01E
:1006A600070E07647FEF03F0075E0450096E046AC5
:1006B600074EFEEF03F0070E076466EF03F00AC06D
:1006C60002F040EF04F0030E076471EF03F0075EDB
:1006D60009380F0B096E074EFEEF03F0D89009326A
:1006E600074EFEEF03F0D8900932074EFEEF03F0F7
:1006F600D8900932FEEF03F0030E076490EF03F083
:10070600075E09380F0B096E0438F00B092604380A
:100716000F0B046E074EFEEF03F0D8900432093239
:10072600074EFEEF03F0D89004320932074EFEEF73
:1007360003F0D89004320932FEEF03F0030E07648B
:10074600B8EF03F0075E09380F0B096E0438F00B9B
:10075600092604380F0B046E0538F00B04260538FD
:100766000F0B056E074EFEEF03F0D89005320432EC
:100776000932074EFEEF03F0D890053204320932F3
:10078600074EFEEF03F0D890053204320932FEEF31
:1007960003F0030E0764E9EF03F0075E09380F0B59
:1007A600096E0438F00B092604380F0B046E053861
:1007B600F00B042605380F0B056E0638F00B0526E0
:1007C60006380F0B066E074EFEEF03F0D890063282
:1007D600053204320932074EFEEF03F0D890063296
:1007E600053204320932074EFEEF03F0D890063286
:1007F600053204320932086A000E0EAE0BEF04F021
:10080600091E041E051E061E092A042205220622AA
:1008160009500826045000220550012206500222E3
:100826000EBE22EF04F0D8A031EF04F002320132FE
:1008360000320832033E31EF04F03BEF04F0D8B04B
:1008460036EF04F0000E081E001E011E021E082AC6
:100856000022012202220A7E36EF04F0010E0C6EFF
:1008660068DC42EF04F0020E0C6E63DC42EF04F02B
:10087600040E0C6E3EDC42EF04F0000E0C6E12000D
:080886000B6A0B86FF0E120045
:10088E00086A096A000E07620364CFEF04F0025093
:10089E0006180A6E075003267E0ED8A05DEF04F0F0
:1008AE00035ED8B0D4EF04F061EF04F0035ED8A07D
:1008BE00D9EF04F0028E068E02C00EF001C00BF0CE
:1008CE0000C00DF0005004026F00D0FF0CF001507C
:1008DE0005026F00D0FF00F06F00CCFF08F004029D
:1008EE00F3500C26F4500822000E00220D50050283
:1008FE00F3500C26F4500822000E0022025004027F
:10090E00F3500826F450002202500502016A000E30
:10091E000122F3500026F45001220D500602F3502E
:10092E000826F4500022026A000E012202220B5009
:10093E000602F3500026F4500122000E02220E5041
:10094E000602F3500126F450022202BEB7EF04F065
:10095E0008360036013602360306D8B4D9EF04F055
:10096E00CAEF04F0D880800E08640030000E00221A
:10097E0001220222D8A0CAEF04F002320132003264
:10098E00034AD4EF04F00AAE029E000EDCEF04F030
:10099E00010E95EC00F0DCEF04F0020E7CEC00F0A2
:0C09AE00DCEF04F0040E88EC00F01200F6
:1009BA000B800BAEE9EF04F0026A0AAEFF0E026E7C
:0C09CA00016E006E0A360232FF0E1200B1
:0609D600067E46DD120062
:1009DC0003500718D8A402EF05F002500618D8A44B
:1009EC0002EF05F001500518D8A402EF05F00050F5
:0E09FC000418D8B4D8841200D8941200120047
:100A0A000450000A12E10550000A0FE10650000ADC
:100A1A000CE10750000A09E1FF0E006EFF0E016E9D
:100A2A007F0E026EFF0E036EA7D0086A096A07508E
:100A3A00D8B4B0EF05F00350D8B4B4EF05F00250C3
:100A4A0006180A6E028E068E0E6A02C008F001C0EF
:100A5A000CF000C00DF004500D5E0550D8A0053C06
:100A6A000C5E0650D8A0063C085E086A0C6A0D6A3D
:100A7A00D8A047EF05F0D89002320132003208328E
:100A8A00010E0E6E0750035ED8A054EF05F07E0EDD
:100A9A000E240326D8B0B9EF05F05AEF05F07E0E02
:100AAA000E240326D8A0BEEF05F0180E0B6E0D36E5
:100ABA000C3608360036013602360E360450005E11
:100ACA000550D8A0053C015E0650D8A0063C025E3F
:100ADA0006340E120EA075EF05F00D8080EF05F0BA
:100AEA00045000260550D8B0053C01260650D8B05F
:100AFA00062802260D900B2E5CEF05F0A6EF05F0F6
:100B0A00D8900036013602360E360450005E055083
:100B1A00D8A0053C015E0650D8A0063C025E063409
:100B2A000E10010B0D26D8B00C2AD8B4082AD8A466
:100B3A00A6EF05F008320C320D32032AD8B4B9EF09
:100B4A0005F00AAE089E0850026E0C50016E0D5058
:100B5A00006EC1EF05F0010E91DEC1EF05F0020E45
:100B6A0095EC00F0C1EF05F0040E7CEC00F0C1EF4B
:0A0B7A0005F0080E88EC00F01200F0
:100B84000050086E0150006E0250016E0350026E58
:100B9400036A0B6A0C6A9E0E036E0A6A020E0C6EDE
:060BA4009CEC00F01200C1
:100BAA000101F751390806E3300EF75D03E3010E40
:080BBA00006E01D0006A120078
:100BC2000A6A0350D8A40A800750D8A40A820A509D
:100BD200D8B444EF06F0030AD8B4FDEF05F00AB02A
:100BE200F8EF05F006AE42EF06F040EF06F002AE77
:100BF20040EF06F042EF06F00250800B0A6E029EB2
:100C02000650800B069E0A18D8B40EEF06F00A5062
:100C1200D8B440EF06F042EF06F00750035CD8B4B8
:100C220018EF06F0D8A034EF06F03AEF06F00650BF
:100C3200025CD8B422EF06F0D8A034EF06F03AEF07
:100C420006F00550015CD8B42CEF06F0D8A034EFC2
:100C520006F03AEF06F00450005CD8B444EF06F018
:100C6200D8B03AEF06F00A52D8B442EF06F040EF9D
:100C720006F00A52D8B440EF06F042EF06F0D880F0
:0E0C82001200D8901200D880D8841200120000
:100C90000B6A0A6A096A005004026F00D0FF09F06B
:100CA0006F00CCFF08F0015005026F00D0FF0BF081
:100CB0006F00CCFF0AF000500502F3500926F450F3
:100CC0000A22E86A0B2201500402F3500926F4506C
:100CD0000A22E86A0B2208C000F009C001F00AC02D
:080CE00002F00BC003F012004A
:100CE800800E0101F719006E800E000A005CD8B072
:100CF80082D1F7510008016E01C0F7F1800E01188A
:100D0800006E800E6E0A005CD8A0CAD0640E046E15
:100D1800F7C100F09DEC01F0120E0024056E000EE4
:100D280000BEFF0E066E000E062205C000F006C0CB
:100D380001F0000E06BEFF0E026E036E0036009034
:100D48000136023603360036009001360236033685
:100D5800280E0024F66E4D0E0120F76E000E0220BC
:100D6800F86E09006F00D4FFF8F109006F00D4FF96
:100D7800F9F109006F00D4FFFAF109006F00D4FF00
:100D8800FBF1640E046EF7C100F09DEC01F008C0A1
:100D980000F00A0E046E9DEC01F0090E0024056EA9
:100DA800000E00BEFF0E066E000E062205C000F003
:100DB80006C001F0000E06BEFF0E026E036E00367E
:100DC80000900136023603360036009001360236AE
:100DD8000336280E0024F66E4D0E0120F76E000E25
:100DE8000220F86E09006F00D4FF00F009006F00C0
:100DF800D4FF01F009006F00D4FF02F009006F0072
:100E0800D4FF03F0F8C104F0F9C105F0FAC106F007
:100E1800FBC107F038DD00C0F8F101C0F9F102C0EC
:100E2800FAF103C0FBF10A0E046EF7C100F09DEC65
:100E380001F008C000F000C001F0000E00BEFF0E77
:100E4800026E036E046E01360190023603360436D4
:100E580001360190023603360436280E0124F66E58
:100E68004D0E0220F76E000E0320F86E09006F0089
:100E7800D4FF00F009006F00D4FF01F009006F00F3
:100E8800D4FF02F009006F00D4FF03F0F8C104F0AA
:100E9800F9C105F0FAC106F0FBC107F0F4DC2AD26B
:100EA800800E0A0A006E800EF719005C78E20A0EBE
:100EB800046EF7C100F09DEC01F0090E0024056EE8
:100EC800000E00BEFF0E066E000E062205C000F0E2
:100ED80006C001F0000E06BEFF0E026E036E00365D
:100EE800009001360236033600360090013602368D
:100EF8000336280E0024F66E4D0E0120F76E000E04
:100F08000220F86E09006F00D4FFF8F109006F00A5
:100F1800D4FFF9F109006F00D4FFFAF109006F005E
:100F2800D4FFFBF10A0E046EF7C100F09DEC01F04E
:100F380008C000F000C001F0000E00BEFF0E026EF7
:100F4800036E046E0136019002360336043601360C
:100F58000190023603360436280E0124F66E4D0E33
:100F68000220F76E000E0320F86E09006F00D4FF10
:100F780000F009006F00D4FF01F009006F00D4FFF2
:100F880002F009006F00D4FF03F0F8C104F0F9C1C2
:100F980005F0FAC106F0FBC107F075DCABD1F7C16B
:100FA80000F0000EF7BFFF0E016E026E036E0036F2
:100FB80000900136023603360036009001360236BC
:100FC8000336280E0024F66E4D0E0120F76E000E33
:100FD8000220F86E09006F00D4FF00F009006F00CE
:100FE800D4FF01F009006F00D4FF02F009006F0080
:100FF800D4FF03F07FD1800EF719006E800E6E0AC1
:10100800005CD8A0CCD0640E046EF7C100F09DEC53
:1010180001F0120E0024056E000E00BEFF0E066ED3
:10102800000E062205C000F006C001F0000E06BE44
:10103800FF0E026E036E003600900136023603364C
:1010480000360090013602360336B20E0024F66EE2
:101058004F0E0120F76E000E0220F86E09006F0097
:10106800D4FFF8F109006F00D4FFF9F109006F000F
:10107800D4FFFAF109006F00D4FFFBF1640E046E8F
:10108800F7C100F09DEC01F008C000F00A0E046EF4
:101098009DEC01F0090E0024056E000E00BEFF0E47
:1010A800066E000E062205C000F006C001F0000E14
:1010B80006BEFF0E026E036E003600900136023641
:1010C800033600360090013602360336B20E00248D
:1010D800F66E4F0E0120F76E000E0220F86E090022
:1010E8006F00D4FF00F009006F00D4FF01F0090081
:1010F8006F00D4FF02F009006F00D4FF03F0F8C1BD
:1011080004F0F9C105F0FAC106F0FBC107F047EC9D
:1011180004F000C0F8F101C0F9F102C0FAF103C00F
:10112800FBF10A0E046EF7C100F09DEC01F008C057
:1011380000F000C001F0000E00BEFF0E026E036E4C
:10114800046E0136019002360336043601360190EA
:10115800023603360436B20E0124F66E4F0E022014
:10116800F76E000E0320F86E09006F00D4FF00F040
:1011780009006F00D4FF01F009006F00D4FF02F0EE
:1011880009006F00D4FF03F0F8C104F0F9C105F0BD
:10119800FAC106F0FBC107F047EC04F0ABD0800EB3
:1011A8000A0A006E800EF719005C79E20A0E046ED6
:1011B800F7C100F09DEC01F0090E0024056E000E49
:1011C80000BEFF0E066E000E062205C000F006C027
:1011D80001F0000E06BEFF0E026E036E0036009090
:1011E80001360236033600360090013602360336E1
:1011F800B20E0024F66E4F0E0120F76E000E02208C
:10120800F86E09006F00D4FFF8F109006F00D4FFF1
:10121800F9F109006F00D4FFFAF109006F00D4FF5B
:10122800FBF10A0E046EF7C100F09DEC01F008C056
:1012380000F000C001F0000E00BEFF0E026E036E4B
:10124800046E0136019002360336043601360190E9
:10125800023603360436B20E0124F66E4F0E022013
:10126800F76E000E0320F86E09006F00D4FF00F03F
:1012780009006F00D4FF01F009006F00D4FF02F0ED
:1012880009006F00D4FF03F0F8C104F0F9C105F0BC
:10129800FAC106F0FBC107F047EC04F02BD0F7C108
:1012A80000F0000EF7BFFF0E016E026E036E0036EF
:1012B80000900136023603360036009001360236B9
:1012C8000336B20E0024F66E4F0E0120F76E000EA4
:1012D8000220F86E09006F00D4FF00F009006F00CB
:1012E800D4FF01F009006F00D4FF02F009006F007D
:0612F800D4FF03F0120018
:1012FE006000E3F6E1FF6000E7F6E2FF6000DFF773
:10130E00E6FFB6C100F0B7C101F027EC02F0120003
:10131E000B6A0C6A0A6A086A0350D8B417EF0AF00F
:10132E00028E9E0E035E03BEA2EF09F0D8B4A2EFAA
:10133E0009F007EF0AF0036C080E035CD8A0D4EF97
:10134E0009F0036E083600C008F001C000F002C0BC
:10135E0001F0026A080E035CD8A0D4EF09F0036E08
:10136E00083600C008F001C000F0016A080E035CE8
:10137E00D8A0D4EF09F0036E083600C008F0006A5A
:10138E00080E035CD8A0D4EF09F0036E0836086A85
:10139E000350D8A4D890E0EF09F00350D8B4E0EF92
:1013AE0009F0D8900232013200320832032ED8EF03
:1013BE0009F00BBC08A0F1EF09F0D8A0F1EF09F08D
:1013CE00082AD8B4002AD8B4012AD8B4022A02BEF8
:1013DE001BEF0AF00AAE17EF0AF0021E011E001EE6
:1013EE00081E082AD8B4002AD8B4012AD8B4022A72
:1013FE0017EF0AF0026A016A006A086A17EF0AF02C
:10140E000B800BAE21EF0AF0026A0AAE21EF0AF052
:10141E00026E016E006E086E0A36023221EF0AF07D
:10142E00000E0C6A22EF0AF0010E0C6EDDEC04F0D9
:10143E0022EF0AF0FF0E0250036E0150026E0050B2
:08144E00016E0850006E12004F
:101456006E0E0101F75DD8A0D6D0640E046EF7C1FA
:1014660000F0ECEC01F0120E0024056E066A000E88
:10147600062205C000F006C001F0000E06BEFF0EF3
:10148600026E036E003600900136023603360036D1
:101496000090013602360336280E0024F66E4D0EF5
:1014A6000120F76E000E0220F86E09006F00D4FFCF
:1014B60000F009006F00D4FF01F009006F00D4FFAF
:1014C60002F009006F00D4FF03F0000E046E000E58
:1014D600056E000E066E7E0E076E47EC04F000C029
:1014E600F8F101C0F9F102C0FAF103C0FBF1640E94
:1014F600046EF7C100F0ECEC01F008C000F00A0E33
:10150600046EECEC01F0090E0024056E066A000E6E
:10151600062205C000F006C001F0000E06BEFF0E52
:10152600026E036E00360090013602360336003630
:101536000090013602360336280E0024F66E4D0E54
:101546000120F76E000E0220F86E09006F00D4FF2E
:1015560000F009006F00D4FF01F009006F00D4FF0E
:1015660002F009006F00D4FF03F0F8C104F0F9C1DE
:1015760005F0FAC106F0FBC107F047EC04F000C025
:10158600F8F101C0F9F102C0FAF103C0FBF10A0E4D
:10159600046EF7C100F0ECEC01F008C000F000C0EA
:1015A60001F0000E026E036E046E013601900236E3
:1015B6000336043601360190023603360436280E09
:1015C6000124F66E4D0E0220F76E000E0320F86E13
:1015D60009006F00D4FF00F009006F00D4FF01F08E
:1015E60009006F00D4FF02F009006F00D4FF03F07A
:1015F600F8C104F0F9C105F0FAC106F0FBC107F025
:1016060047EC04F0BDD0F7510A08D8B086D00A0ED0
:10161600046EF7C100F0ECEC01F0090E0024056E33
:10162600066A000E062205C000F006C001F0000E94
:1016360006BEFF0E026E036E0036009001360236BD
:10164600033600360090013602360336280E002493
:10165600F66E4D0E0120F76E000E0220F86E0900A0
:101666006F00D4FF00F009006F00D4FF01F00900FD
:101676006F00D4FF02F009006F00D4FF03F0000EE4
:10168600046E000E056E000E066E7E0E076E47ECAB
:1016960004F000C0F8F101C0F9F102C0FAF103C08C
:1016A600FBF10A0E046EF7C100F0ECEC01F008C085
:1016B60000F000C001F0000E026E036E046E0136EB
:1016C600019002360336043601360190023603369F
:1016D6000436280E0124F66E4D0E0220F76E000E1B
:1016E6000320F86E09006F00D4FF00F009006F00B8
:1016F600D4FF01F009006F00D4FF02F009006F006B
:10170600D4FF03F0F8C104F0F9C105F0FAC106F000
:10171600FBC107F047EC04F033D0F7C100F0000E30
:10172600016E026E036E00360090013602360336F5
:1017360000360090013602360336280E0024F66E77
:101746004D0E0120F76E000E0220F86E09006F00A4
:10175600D4FF00F009006F00D4FF01F009006F000C
:10176600D4FF02F009006F00D4FF03F0000E046EF0
:10177600000E056E000E066E7E0E076E47EC04F038
:0217860012004F
:101788000450000A08E10550000A05E1FF0E006E4A
:101798007F0E016E58D00D6A096A086A0150001060
:1017A800D8B4000C015005180A6E0ABE0D1E0B6A4B
:1017B80005AE05D0041E051E042AD8B4052A01AEBC
:1017C80005D0001E011E002AD8B4012A01500510B8
:1017D8000A6E0ABE10D0FBEC01F00BB020D00DAEA3
:1017E800000C001E011E002AD8B4012A081E091E7A
:1017F800082AD8B4092A000C05AE0DD001BE07D0BE
:101808000150096E0050086E016A006AE8D7016A43
:10181800006A002A000C011E001E0B2ADDD7082AC8
:10182800D8B4092A0450085CD8A4D9D70550095C53
:10183800D8A4D5D7096A086A002AD8B4012A01AE03
:08184800CED70000FF0C1200D6
:101850000B6A0A6A096A086A0E6A03340836045079
:10186000085E0550D8A0053C095E0650D8A0063C8D
:101870000A5E0750D8A0073C0B5EE86AD8A0010EAC
:101880000E5E0336070E0C6E0334083609360A3630
:101890000B360E36045003A012D0085E0550D8A0B7
:1018A000053C095E0650D8A0063C0A5E0750D8A049
:1018B000073C0B5EE86AD8A0010E0E5E11D0082628
:1018C0000550D8B0053C09260650D8B0063C0A267B
:1018D0000750D8B0073C0B26E86AD8B0010E0E2698
:1018E00003360C2ED1D70234083609360A360B36A9
:1018F0000E36045003A012D0085E0550D8A0053C57
:10190000095E0650D8A0063C0A5E0750D8A0073CE6
:101910000B5EE86AD8A0010E0E5E11D008260550B5
:10192000D8B0053C09260650D8B0063C0A26075018
:10193000D8B0073C0B26E86AD8B0010E0E26023656
:10194000070E0C6E0234083609360A360B360E3690
:10195000045002A012D0085E0550D8A0053C095ED4
:101960000650D8A0063C0A5E0750D8A0073C0B5E84
:10197000E86AD8A0010E0E5E11D008260550D8B036
:10198000053C09260650D8B0063C0A260750D8B0B8
:10199000073C0B26E86AD8B0010E0E2602360C2E44
:1019A000D1D70134083609360A360B360E360450C4
:1019B00002A012D0085E0550D8A0053C095E065072
:1019C000D8A0063C0A5E0750D8A0073C0B5EE86A28
:1019D000D8A0010E0E5E11D008260550D8B0053CE7
:1019E00009260650D8B0063C0A260750D8B0073C56
:1019F0000B26E86AD8B0010E0E260136070E0C6ED3
:101A00000134083609360A360B360E36045001A06A
:101A100012D0085E0550D8A0053C095E0650D8A03B
:101A2000063C0A5E0750D8A0073C0B5EE86AD8A0C7
:101A3000010E0E5E11D008260550D8B0053C0926CF
:101A40000650D8B0063C0A260750D8B0073C0B26F3
:101A5000E86AD8B0010E0E2601360C2ED1D700341C
:101A6000083609360A360B360E36045001A012D05D
:101A7000085E0550D8A0053C095E0650D8A0063C7B
:101A80000A5E0750D8A0073C0B5EE86AD8A0010E9A
:101A90000E5E11D008260550D8B0053C0926065028
:101AA000D8B0063C0A260750D8B0073C0B26E86A97
:101AB000D8B0010E0E260036070E0C6E0034083624
:101AC00009360A360B360E36045000A012D0085ED6
:101AD0000550D8A0053C095E0650D8A0063C0A5E19
:101AE0000750D8A0073C0B5EE86AD8A0010E0E5E36
:101AF00011D008260550D8B0053C09260650D8B0AC
:101B0000063C0A260750D8B0073C0B26E86AD8B036
:101B1000010E0E2600360C2ED1D700B00ED0045088
:101B200008260550D8B0053C09260650D8B0063C1A
:0C1B30000A260750D8B0073C0B26120014
:101B3C000B6A0C6A086A0350D8B422EF0EF002C08C
:101B4C000AF0028E9E0E035E03AE12EF0EF0036CD3
:101B5C00080E035CD8A0DFEF0DF0036E083600C052
:101B6C0008F001C000F002C001F0026A080E035C2C
:101B7C00D8A0DFEF0DF0036E083600C008F001C0EE
:101B8C0000F0016A080E035CD8A0DFEF0DF0036EC5
:101B9C00083600C008F0006A080E035CD8A0DFEF1E
:101BAC000DF0036E0836086A0350D8A4D890EBEFFA
:101BBC000DF00350D8B4EBEF0DF0D8900232013297
:101BCC0000320832032EE3EF0DF00BBC08A0FCEF43
:101BDC000DF0D8A0FCEF0DF0082AD8B4002AD8B428
:101BEC00012AD8B4022A02BE26EF0EF00AAE22EF6A
:101BFC000EF0021E011E001E081E082AD8B4002A70
:101C0C00D8B4012AD8B4022A22EF0EF0026A016A73
:101C1C00006A086A22EF0EF00B800BAE2DEF0EF06F
:101C2C00026A0AAE2DEF0EF0026E016E006E086EA7
:101C3C000A3602322DEF0EF00C6A000E2EEF0EF06B
:101C4C00010E0C6E000EDDEC04F02EEF0EF0FF0E0C
:101C5C000250036E0150026E0050016E0850006E6F
:021C6C00120064
:101C6E000101EF6BF06BE36BE46BD1C100F0D2C1FD
:101C7E0001F0D3C102F0010ED127000ED223D323DF
:101C8E00600003F0F6FF600007F0F7FF60000BF056
:101C9E00F8FF09006F00D4FF00F000C0E0F1005221
:101CAE00D8B4B6EF1FF0E051250A0EE060003FF702
:101CBE00E1FF600043F7E2FF600083F7E6FFCF4BE2
:101CCE00D02BEF4BF02BD1D7E16BE26BE36BE46BD8
:101CDE0023D0E387010ED127000ED223D3236DD05C
:101CEE00E381010ED127000ED223D32366D0E383E6
:101CFE00010ED127000ED223D3235FD0E487010E2D
:101D0E00D127000ED223D32358D0E385010ED1273D
:101D1E00000ED223D32351D0600047F7F6FF6000A8
:101D2E004BF7F7FF60004FF7F8FF09006F00D4FF85
:101D3E0001F001502D0ACDE0600047F7F6FF60007C
:101D4E004BF7F7FF60004FF7F8FF09006F00D4FF65
:101D5E0001F00150200AC4E0600047F7F6FF600072
:101D6E004BF7F7FF60004FF7F8FF09006F00D4FF45
:101D7E0001F001502B0ABBE0600047F7F6FF600050
:101D8E004BF7F7FF60004FF7F8FF09006F00D4FF25
:101D9E0001F00150230AB2E0600047F7F6FF600041
:101DAE004BF7F7FF60004FF7F8FF09006F00D4FF05
:101DBE0001F00150300AA9E001D08AD7E3A301D087
:101DCE00E391E3A701D0E395600047F7F6FF6000CB
:101DDE004BF7F7FF60004FF7F8FF09006F00D4FFD5
:101DEE0000F0000E016E00C0F7F1D5EC05F00052C8
:101DFE003EE0E16BE26BE1C100F0E2C101F00A0EE0
:101E0E00046E000E056E48EC06F0600047F7F6FF14
:101E1E0060004BF7F7FF60004FF7F8FF09006F0007
:101E2E00D4FF02F002500024E16F000E0120E26F99
:101E3E00300EE15F000EE25B010ED127000ED223C1
:101E4E00D323600047F7F6FF60004BF7F7FF600003
:101E5E004FF7F8FF09006F00D4FF00F0000E016E7F
:101E6E0000C0F7F1D5EC05F00052C5E145D0600099
:101E7E0047F7F6FF60004BF7F7FF60004FF7F8FFEC
:101E8E0009006F00D4FF01F001502A0A35E160000D
:101E9E0053F7E9FF600057F7EAFF6F00B8FF00F055
:101EAE006F00B8FF01F0600003F0E9FF600007F07B
:101EBE00EAFF6F00B8FFE1F16F00B8FFE2F16000DA
:101ECE0053F7E9FF600057F7EAFF020EEE24006EAB
:101EDE00000EEE20016E600053F7E1FF600057F731
:101EEE00E2FF600003F0E6FF600007F0E6FF010E80
:101EFE00D127000ED223D323600047F7F6FF6000F0
:101F0E004BF7F7FF60004FF7F8FF09006F00D4FFA3
:101F1E0001F001502E0AD8A48AD0010ED127000E4E
:101F2E00D223D323600047F7F6FF60004BF7F7FF8D
:101F3E0060004FF7F8FF09006F00D4FF01F0015069
:101F4E002A0A36E1600053F7E9FF600057F7EAFF0F
:101F5E006F00B8FF00F06F00B8FF01F0600003F0F3
:101F6E00E9FF600007F0EAFF6F00B8FFDEF16F00D7
:101F7E00B8FFDFF1600053F7E9FF600057F7EAFFA3
:101F8E00020EEE24006E000EEE20016E600053F77E
:101F9E00E1FF600057F7E2FF600003F0E6FF60002C
:101FAE0007F0E6FF010ED127000ED223D3233ED039
:101FBE00DE6BDF6B600047F7F6FF60004BF7F7FF55
:101FCE0060004FF7F8FF09006F00D4FF00F0000E1D
:101FDE00016E00C0F7F1D5EC05F0005227E0DEC12E
:101FEE0000F0DFC101F00A0E046E000E056E48EC23
:101FFE0006F0600047F7F6FF60004BF7F7FF600052
:10200E004FF7F8FF09006F00D4FF02F002500024D2
:10201E00DE6F000E0120DF6F300EDE5F000EDF5B25
:10202E00010ED127000ED223D323C4D703D0DE6BEB
:10203E00DF6BE489D1C100F0D2C101F0D3C102F04F
:10204E00010ED127000ED223D323600003F0F6FF3A
:10205E00600007F0F7FF60000BF0F8FF09006F005B
:10206E00D4FFE0F11DD1EFC100F0F0C101F0BAEFE5
:10207E001FF0E389DFD7E48552D1E38BE4814FD1A2
:10208E00E4834DD1E38D4BD14AD1E38BE38F47D11E
:10209E00600053F7E9FF600057F7EAFF6F00B8FFE3
:1020AE0000F06F00B8FF01F0600003F0E9FF600080
:1020BE0007F0EAFF6F00B8FFEBF16F00B8FFECF12D
:1020CE00600053F7E9FF600057F7EAFF020EEE24B7
:1020DE00006E000EEE20016E600053F7E1FF60000F
:1020EE0057F7E2FF600003F0E6FF600007F0E6FF3F
:1020FE00000EEC1902E1000EEB1904E1400EEB6F3D
:10210E00000EEC6FED6BEE6BED51EB25E96EEE51C3
:10211E00EC21EA6EEE520BE0010EED25006E000E84
:10212E00EE21016E00C0EDF101C0EEF1EDD7DE51F2
:10213E00DF110AE0EE51DF5D02E1ED51DE5D04E2FA
:10214E00DEC1EDF1DFC1EEF1E251EE5D02E1E151F2
:10215E00ED5D05E2ED51E15FEE51E25B02D0E16B28
:10216E00E26BE3B718D0E1C100F0E2C101F0010E5D
:10217E00E15F000EE25B005001100DE060003FF7E2
:10218E00E1FF600043F7E2FF200EE66ECF4BD02B4F
:10219E00EF4BF02BE8D7EDC102F0EEC103F0010ECC
:1021AE00ED5D006E000EEE59016E00C0EDF101C046
:1021BE00EEF1025003101EE06000AFF7E9FF600081
:1021CE00B3F7EAFF60003FF7E1FF600043F7E2FF7D
:1021DE006F00BBFFE6FFCF4BD02B010EEB25006E41
:1021EE00000EEC21016E00C0EBF101C0ECF1EF4BE3
:1021FE00F02BD1D7E3A718D0E1C100F0E2C101F076
:10220E00010EE15F000EE25B005001100DE0600078
:10221E003FF7E1FF600043F7E2FF200EE66ECF4B83
:10222E00D02BEF4BF02BE8D720D5600053F7E9FF0A
:10223E00600057F7EAFF6F00B8FF00F06F00B8FFBD
:10224E0001F0600003F0E9FF600007F0EAFF6F00A5
:10225E00B8FFE0F1600053F7E9FF600057F7EAFFBF
:10226E00020EEE24006E000EEE20016E600053F79B
:10227E00E1FF600057F7E2FF600003F0E6FF600049
:10228E0007F0E6FFE00EEB6F010EEC6F010EED6F47
:10229E00000EEE6F4CD7C00EE313000EE4133FD0CA
:1022AE00E051000AD8B4DFD6E0516C0AD8B4E1D6BA
:1022BE00E0514C0AD8B4DDD6E051660AD8B4DBD66C
:1022CE00E051450AD8B4D9D6E051650AD8B4D6D66D
:1022DE00E051670AD8B4D4D6E0516F0AD8B4D2D63A
:1022EE00E051640AD8B4D0D6E051690AD8B4CCD63D
:1022FE00E051700AD8B4C9D6E051580AD8B4C5D640
:10230E00E051780AD8B4C2D6E051730AD8B4C0D618
:10231E00E051630A8AE0E051750ABDE0B3D7000EC2
:10232E00E315006EE451070B016E00500110D8B496
:10233E00E1EF1AF0E4A904D0060EDE6F000EDF6F97
:10234E00600053F7E9FF600057F7EAFF6F00B8FF30
:10235E0000F06F00B8FF01F0600003F0E9FF6000CD
:10236E0007F0EAFF6F00B8FFE5F16F00B8FFE6F186
:10237E006F00B8FFE7F16F00B8FFE8F1600053F7A8
:10238E00E9FF600057F7EAFF040EEE24006E000E20
:10239E00EE20016E600053F7E1FF600057F7E2FF99
:1023AE00600003F0E6FF600007F0E6FF046A056ACE
:1023BE00066A076AE5C100F0E6C101F0E7C102F066
:1023CE00E8C103F0E1EC05F0010ED8B0000E006E8E
:1023DE00005205E0E77F030EE313000EE413E96BF2
:1023EE00EA6BE5C100F0E6C101F0E7C102F0E8C119
:1023FE0003F0046A056A066A076AEEEC04F0000E42
:10240E00D8A4010E006E0052D8B48AD0E8C100F0F4
:10241E00016A026A036AFF0E0016000E01167E0E96
:10242E00005E000E015A00C0E9F101C0EAF1010E92
:10243E00005E000E015A00C0E9F101C0EAF1030E80
:10244E00046E000E056E48EC06F000C0E9F101C006
:10245E00EAF10A0E046E000E056EC4EC0BF000C01D
:10246E00E9F101C0EAF1800E0118026E800E025CE5
:10247E0002E1000E005C05E2010E0101E95F000EB3
:10248E00EA5B0101E9510008F76F74EC06F0E5C153
:10249E0004F0E6C105F0E7C106F0E8C107F047EC2D
:1024AE0004F000C0EBF101C0ECF102C0EDF103C08D
:1024BE00EEF1000E046E000E056E000E066E7F0E1F
:1024CE00076EEBC100F0ECC101F0EDC102F0EEC100
:1024DE0003F0E1EC05F0010ED8B0000E006E0052D4
:1024EE0005E0010EE95F000EEA5B1AD0000E046EE5
:1024FE00000E056E200E066E820E076EEBC100F00A
:10250E00ECC101F0EDC102F0EEC103F0E1EC05F01B
:10251E00000ED8B0010E006E005202E0E94BEA2B1D
:10252E00800E006E800EEA19005C02E1E95100088F
:10253E0003E3010EE06F02D0E9C1E0F1E4B119D07E
:10254E00E4A315D0800EEA19006E7F0E005C02E146
:10255E00FC0EE95D0BE3800EEA19006E800EDF19AA
:10256E00005C02E1DE51E95D01E201D002D0E7EF4D
:10257E0016F0DE51DF1106E0E4A304D0010EDE5F9B
:10258E00000EDF5BDF51000802E1DE51080803E2B6
:10259E00080EE06F02D0DEC1E0F1E5C100F0E6C149
:1025AE0001F0E7C102F0E8C103F0046A056A066AA9
:1025BE00076AEEEC04F0000ED8A4010E006E005275
:1025CE00D8B453D1E9C1F7F174EC06F000C004F0B1
:1025DE0001C005F002C006F003C007F0E5C100F02F
:1025EE00E6C101F0E7C102F0E8C103F005EC05F029
:1025FE0000C0E5F101C0E6F102C0E7F103C0E8F169
:10260E000101E0510008F76F74EC06F000C004F011
:10261E0001C005F002C006F003C007F0E5C100F0EE
:10262E00E6C101F0E7C102F0E8C103F005EC05F0E8
:10263E0000C0F1F101C0F2F102C0F3F103C0F4F1F8
:10264E00F1C1E5F1F2C1E6F1F3C1E7F1F4C1E8F150
:10265E00F1C100F0F2C101F0F3C102F0F4C103F0D8
:10266E008FEC09F0C2EC05F000C004F001C005F0DB
:10267E0002C006F003C007F0F1C100F0F2C101F094
:10268E00F3C102F0F4C103F0EBEC04F0000E046EA3
:10269E00000E056E000E066E7E0E076EE1EC05F066
:1026AE00000ED8B0010E006E00521AE0E5C100F027
:1026BE00E6C101F0E7C102F0E8C103F0000E046EBE
:1026CE00000E056E000E066E7E0E076E33EC02F0E7
:1026DE0000C0E5F101C0E6F102C0E7F103C0E8F188
:1026EE00E5C100F0E6C101F0E7C102F0E8C103F078
:1026FE008FEC09F00101E051010F096E0A6A000E1C
:10270E000A2209C004F00AC005F0000E0ABEFF0E30
:10271E00066E076E04360490053606360736043606
:10272E000490053606360736410E0424F66E500E1A
:10273E000520F76E000E0620F86E09006F00D4FF1C
:10274E0005F009006F00D4FF06F009006F00D4FFFA
:10275E0007F009006F00D4FF08F00850035C08E191
:10276E000750025C05E10650015C02E10550005C79
:10277E001EE30101E5C100F0E6C101F0E7C102F080
:10278E00E8C103F0CD0E046ECC0E056E4C0E066E37
:10279E007B0E076E47EC04F000C0E5F101C0E6F1D8
:1027AE0002C0E7F103C0E8F1E94BEA2B5ED0E5C1C8
:1027BE0000F0E6C101F0E7C102F0E8C103F08FECD2
:1027CE0009F0E0C104F0000E056E066E076E0436C9
:1027DE00049005360636073604360490053606365E
:1027EE000736410E0424F66E500E0520F76E000ECD
:1027FE000620F86E09006F00D4FF05F009006F0087
:10280E00D4FF06F009006F00D4FF07F009006F0037
:10281E00D4FF08F00850035C08E10750025C05E1A4
:10282E000650015C02E10550005C1FE20101E5C1AA
:10283E0000F0E6C101F0E7C102F0E8C103F0000EBE
:10284E00046E000E056E200E066E820E076E47ECAD
:10285E0004F000C0E5F101C0E6F102C0E7F103C0EB
:10286E00E8F1010EE95F000EEA5B0101E4A393D0EB
:10287E00E4B791D0800E000A006E800EDF19005C66
:10288E0002E1DE510A0804E20A0EDE6F000EDF6F6F
:10289E00E5C100F0E6C101F0E7C102F0E8C103F0C6
:1028AE008FEC09F000C0EBF101C0ECF102C0EDF1CC
:1028BE0003C0EEF1EB51EC11ED11EE1142E00A0EF8
:1028CE00046E000E056E066E076EEBC100F0ECC1D5
:1028DE0001F0EDC102F0EEC103F028EC0CF008C0DF
:1028EE0000F009C001F00AC002F00BC003F0000EA8
:1028FE00046E031808E10450021805E10450011893
:10290E0002E10050000A1DE1010EDE5F000EDF5BEA
:10291E000A0E046E000E056E066E076EEBC100F019
:10292E00ECC101F0EDC102F0EEC103F028EC0CF0A9
:10293E0000C0EBF101C0ECF102C0EDF103C0EEF10D
:10294E00B9D7800EDF19006E800E005C02E1E051F7
:10295E00DE5D21E2DE51E05DF76F74EC06F000C043
:10296E0004F001C005F002C006F003C007F0E5C197
:10297E0000F0E6C101F0E7C102F0E8C103F005EC9A
:10298E0005F000C0E5F101C0E6F102C0E7F103C0B9
:10299E00E8F1DEC1E0F1050E0101DE25006E000E4C
:1029AE00DF21016E0050E15F0150E25BDE51DF116D
:1029BE0003E1E4B701D004D0010EE15F000EE25B4B
:1029CE00030EE315006EE4C101F0000E0116005077
:1029DE00011004E0010EE15F000EE25BE3A540D0C2
:1029EE00E3A315D0E3A103D02D0ED66F02D02B0E8C
:1029FE00D66F60003FF7E1FF600043F7E2FF600033
:102A0E005BF7E6FFCF4BD02BEF4BF02B0ED0E3A1B5
:102A1E000CD060003FF7E1FF600043F7E2FF200EAD
:102A2E00E66ECF4BD02BEF4BF02B800E006E800E50
:102A3E00E219005C02E1E151000811E260003FF78B
:102A4E00E1FF600043F7E2FF300EE66ECF4BD02B76
:102A5E00EF4BF02B010EE15F000EE25BE6D741D0AB
:102A6E00E3B71AD0800E006E800EE219005C02E110
:102A7E00E151000811E260003FF7E1FF600043F70B
:102A8E00E2FF200EE66ECF4BD02BEF4BF02B010E5C
:102A9E00E15F000EE25BE6D7E3A315D0E3A103D01E
:102AAE002D0ED76F02D02B0ED76F60003FF7E1FFD0
:102ABE00600043F7E2FF60005FF7E6FFCF4BD02BDD
:102ACE00EF4BF02B0ED0E3A10CD060003FF7E1FFEF
:102ADE00600043F7E2FF200EE66ECF4BD02BEF4B9C
:102AEE00F02BE5C100F0E6C101F0E7C102F0E8C14C
:102AFE0003F08FEC09F000C0EBF101C0ECF102C065
:102B0E00EDF103C0EEF1E0C100F0000E016E026EB9
:102B1E00036E003600900136023603360036009002
:102B2E00013602360336410E0024F66E500E012099
:102B3E00F76E000E0220F86E09006F00D4FF04F04D
:102B4E0009006F00D4FF05F009006F00D4FF06F0F6
:102B5E0009006F00D4FF07F0EBC100F0ECC101F0EB
:102B6E00EDC102F0EEC103F028EC0CF0300E0026A1
:102B7E0060003FF7E1FF600043F7E2FF600003F003
:102B8E00E6FFCF4BD02BEF4BF02BDE51DF1103E1E5
:102B9E00E4B701D07AD060003FF7E1FF600043F761
:102BAE00E2FF2E0EE66ECF4BD02BEF4BF02BE0510B
:102BBE00DE5F000EDF5BE05354E0E007E0C100F0A3
:102BCE00000E016E026E036E003600900136023664
:102BDE00033600360090013602360336410E0024CD
:102BEE00F66E500E0120F76E000E0220F86E0900F0
:102BFE006F00D4FF04F009006F00D4FF05F0090048
:102C0E006F00D4FF06F009006F00D4FF07F0EBC190
:102C1E0000F0ECC101F0EDC102F0EEC103F028ECC2
:102C2E000CF00A0E046E000E056E066E076E28EC92
:102C3E000CF008C000F009C001F00AC002F00BC091
:102C4E0003F0300E002660003FF7E1FF600043F70F
:102C5E00E2FF600003F0E6FFCF4BD02BEF4BF02BE3
:102C6E00AAD7DE51DF1111E060003FF7E1FF6000EF
:102C7E0043F7E2FF300EE66ECF4BD02BEF4BF02B2F
:102C8E00010EDE5F000EDF5BECD7E3AB0DD0600014
:102C9E003FF7E1FF600043F7E2FF450EE66ECF4BD4
:102CAE00D02BEF4BF02B0CD060003FF7E1FF600014
:102CBE0043F7E2FF650EE66ECF4BD02BEF4BF02BBA
:102CCE00800EEA19006E800E005C02E1000EE95DD6
:102CDE0013E2E9510008E96FEA51000EEA5760006D
:102CEE003FF7E1FF600043F7E2FF2D0EE66ECF4B9C
:102CFE00D02BEF4BF02B0CD060003FF7E1FF6000C4
:102D0E0043F7E2FF2B0EE66ECF4BD02BEF4BF02BA3
:102D1E000A0E046E000E056EE9C100F0EAC101F064
:102D2E00C4EC0BF0300E002660003FF7E1FF6000B0
:102D3E0043F7E2FF600003F0E6FF0101CF4BD02B1B
:102D4E00EF4BF02B0A0E046E000E056EE9C100F07B
:102D5E00EAC101F0C4EC0BF008C000F009C001F0AC
:102D6E00300E002660003FF7E1FF600043F7E2FF00
:102D7E00600003F0E6FF0101CF4BD02BEF4BF02BA1
:102D8E00E3A71CD0800E006E800EE219005C02E1FB
:102D9E00E151000813E260003FF7E1FF600043F7E6
:102DAE00E2FF200EE66ECF4BD02BEF4BF02B010E39
:102DBE00E15F000EE25BE151E211EDE13CEF0EF05E
:102DCE00E4A3F7D0800EEA19006E800E005C02E1DB
:102DDE00000EE95D0AE2010EE95D006E000EEA5991
:102DEE00016E0050DE5F0150DF5BE5C100F0E6C111
:102DFE0001F0E7C102F0E8C103F08FEC09F000C06A
:102E0E00EBF101C0ECF102C0EDF103C0EEF1010EE9
:102E1E00E06FE0510A0A38E0E0C100F0000E016EEA
:102E2E00026E036E0036009001360236033600360F
:102E3E000090013602360336410E0024F66E500E17
:102E4E000120F76E000E0220F86E09006F00D4FF0D
:102E5E0001F009006F00D4FF02F009006F00D4FFEB
:102E6E0003F009006F00D4FF04F00450EE5D08E19A
:102E7E000350ED5D05E10250EC5D02E10150EB5DAA
:102E8E0001E202D0E02BC5D7E051DE5DF56F000EFA
:102E9E00DF59F66FF5C1DEF1F6C1DFF1EBC100F0DF
:102EAE00ECC101F0EDC102F0EEC103F0C2EC05F091
:102EBE0000C004F001C005F002C006F003C007F028
:102ECE00E5C100F0E6C101F0E7C102F0E8C103F090
:102EDE00EBEC04F000C0F1F101C0F2F102C0F3F12D
:102EEE0003C0F4F1F5C1F7F174EC06F0F1C104F092
:102EFE00F2C105F0F3C106F0F4C107F047EC04F09F
:102F0E00000E046E000E056E000E066E7E0E076E2F
:102F1E0033EC02F08FEC09F000C0EBF101C0ECF1E4
:102F2E0002C0EDF103C0EEF1DE51DF1142E00A0EF8
:102F3E00046E000E056E066E076EEBC100F0ECC15E
:102F4E0001F0EDC102F0EEC103F028EC0CF008C068
:102F5E0000F009C001F00AC002F00BC003F0000E31
:102F6E00046E031808E10450021805E1045001181C
:102F7E0002E10050000A1DE10A0E046E000E056EFD
:102F8E00066E076EEBC100F0ECC101F0EDC102F070
:102F9E00EEC103F028EC0CF000C0EBF101C0ECF137
:102FAE0002C0EDF103C0EEF1010EDE5F000EDF5B3D
:102FBE00BBD7800E006E800EDF19005C02E1DE5181
:102FCE000C0816E3DEC1F7F12BEC0AF0E5C104F0B4
:102FDE00E6C105F0E7C106F0E8C107F033EC02F0F8
:102FEE0000C0E5F101C0E6F102C0E7F103C0E8F16F
:102FFE00E5C100F0E6C101F0E7C102F0E8C103F05F
:10300E00046A056A066A076AEEEC04F0000ED8A49C
:10301E00010E006E0052D8B477D0E5C100F0E6C1C3
:10302E0001F0E7C102F0E8C103F08FEC09F0000EE9
:10303E00046E031808E10450021805E1045001184B
:10304E0002E10050000A60E1800E006E800EEA1967
:10305E00005C02E1E951010857E2E9C1F7F174ECB5
:10306E0006F000C004F001C005F002C006F003C077
:10307E0007F0E5C100F0E6C101F0E7C102F0E8C1DA
:10308E0003F005EC05F05F0E046E700E056E090E72
:10309E00066E810E076EE1EC05F0010ED8B0000E43
:1030AE00006E005206E0090E0101E95F000EEA5BB8
:1030BE0005D00101080EE95F000EEA5BE9C1F7F1E8
:1030CE0074EC06F000C004F001C005F002C006F07A
:1030DE0003C007F0E5C100F0E6C101F0E7C102F060
:1030EE00E8C103F005EC05F08FEC09F000C0EBF140
:1030FE0001C0ECF102C0EDF103C0EEF10101E56B90
:10310E00E66BE76BE86B38D0E5C100F0E6C101F085
:10311E00E7C102F0E8C103F08FEC09F000C0EBF15B
:10312E0001C0ECF102C0EDF103C0EEF1EBC100F015
:10313E00ECC101F0EDC102F0EEC103F0C2EC05F0FE
:10314E0000C004F001C005F002C006F003C007F095
:10315E00E5C100F0E6C101F0E7C102F0E8C103F0FD
:10316E00EBEC04F000C0E5F101C0E6F102C0E7F1BE
:10317E0003C0E8F1E96BEA6B010EE06FE0510A0A59
:10318E0038E0E0C100F0000E016E026E036E0036F4
:10319E0000900136023603360036009001360236B4
:1031AE000336410E0024F66E500E0120F76E000E0F
:1031BE000220F86E09006F00D4FF01F009006F00C5
:1031CE00D4FF02F009006F00D4FF03F009006F0076
:1031DE00D4FF04F00450EE5D08E10350ED5D05E10F
:1031EE000250EC5D02E10150EB5D01E202D0E02BFA
:1031FE00C5D7E051DE25006E000EDF21016EE951CC
:10320E000026EA5101220050E15F0150E25BE4B773
:10321E0004D0DE51DF1101E104D0010EE15F000E9A
:10322E00E25B030EE315006EE4C101F0000E011621
:10323E000050011004E0010EE15F000EE25BE3A519
:10324E0040D0E3A315D0E3A103D02D0ED86F02D04A
:10325E002B0ED86F60003FF7E1FF600043F7E2FFEF
:10326E00600063F7E6FFCF4BD02BEF4BF02B0ED069
:10327E00E3A10CD060003FF7E1FF600043F7E2FFEF
:10328E00200EE66ECF4BD02BEF4BF02B800E006E48
:10329E00800EE219005C02E1E151000811E26000CB
:1032AE003FF7E1FF600043F7E2FF300EE66ECF4BD3
:1032BE00D02BEF4BF02B010EE15F000EE25BE6D759
:1032CE0041D0E3B71AD0800E006E800EE219005C7A
:1032DE0002E1E151000811E260003FF7E1FF6000FA
:1032EE0043F7E2FF200EE66ECF4BD02BEF4BF02BC9
:1032FE00010EE15F000EE25BE6D7E3A315D0E3A17A
:10330E0003D02D0ED96F02D02B0ED96F60003FF770
:10331E00E1FF600043F7E2FF600067F7E6FFCF4B87
:10332E00D02BEF4BF02B0ED0E3A10CD060003FF76B
:10333E00E1FF600043F7E2FF200EE66ECF4BD02B8D
:10334E00EF4BF02BE0C100F0E007005253E0E0C17C
:10335E0000F0000E016E026E036E00360090013614
:10336E000236033600360090013602360336410E21
:10337E000024F66E500E0120F76E000E0220F86E3D
:10338E0009006F00D4FF04F009006F00D4FF05F0B0
:10339E0009006F00D4FF06F009006F00D4FF07F09C
:1033AE00EBC100F0ECC101F0EDC102F0EEC103F093
:1033BE0028EC0CF00A0E046E000E056E066E076EFB
:1033CE0028EC0CF008C000F009C001F00AC002F0B1
:1033DE000BC003F0300E002660003FF7E1FF6000E7
:1033EE0043F7E2FF600003F0E6FFCF4BD02BEF4B2D
:1033FE00F02BA8D7800E006E800EEA19005C02E159
:10340E00E951000811E260003FF7E1FF600043F769
:10341E00E2FF300EE66ECF4BD02BEF4BF02B010EB2
:10342E00E95F000EEA5BE6D7800E000A006E800EA2
:10343E00DF19005C02E1DE51080803E2080EE06FBE
:10344E0002D0DEC1E0F1E051DE5F000EDF5BE05343
:10345E0003E1E4B701D00CD060003FF7E1FF60005C
:10346E0043F7E2FF2E0EE66ECF4BD02BEF4BF02B39
:10347E00E0C1F7F174EC06F0E5C104F0E6C105F029
:10348E00E7C106F0E8C107F047EC04F09EEC0DF042
:10349E0000C0EBF101C0ECF102C0EDF103C0EEF1A2
:1034AE00E05354E0E007E0C100F0000E016E026E42
:1034BE00036E003600900136023603360036009059
:1034CE00013602360336410E0024F66E500E0120F0
:1034DE00F76E000E0220F86E09006F00D4FF04F0A4
:1034EE0009006F00D4FF05F009006F00D4FF06F04D
:1034FE0009006F00D4FF07F0EBC100F0ECC101F042
:10350E00EDC102F0EEC103F028EC0CF00A0E046ED1
:10351E00000E056E066E076E28EC0CF008C000F06B
:10352E0009C001F00AC002F00BC003F0300E0026F5
:10353E0060003FF7E1FF600043F7E2FF600003F039
:10354E00E6FFCF4BD02BEF4BF02BAAD7DE51DF117E
:10355E0011E060003FF7E1FF600043F7E2FF300E3D
:10356E00E66ECF4BD02BEF4BF02B010EDE5F000E35
:10357E00DF5BECD7E3A71CD0800E006E800EE21945
:10358E00005C02E1E151000813E260003FF7E1FF49
:10359E00600043F7E2FF200EE66ECF4BD02BEF4BD1
:1035AE00F02B010EE15F000EE25BE151E211EDE165
:1035BE003CEF0EF0C00EE315016EE4C102F0000EFA
:1035CE000216000E021802E1000E0118D8A49ED0B9
:1035DE00E3A937D0600053F7E9FF600057F7EAFF21
:1035EE006F00B8FF00F06F00B8FF01F0600003F04D
:1035FE00E9FF600007F0EAFF6F00B8FFEBF16F0024
:10360E00B8FFECF16F00B8FFEDF16F00B8FFEEF10F
:10361E00600053F7E9FF600057F7EAFF040EEE244F
:10362E00006E000EEE20016E600053F7E1FF6000A9
:10363E0057F7E2FF600003F0E6FF600007F0E6FFD9
:10364E003DD0600053F7E9FF600057F7EAFF6F00C7
:10365E00B8FF00F06F00B8FF01F0600003F0E9FF63
:10366E00600007F0EAFF6F00B8FF00F06F00B8FFD0
:10367E0001F0000E01BEFF0E026E036E00C0EBF1F4
:10368E0001C0ECF102C0EDF103C0EEF1600053F7A2
:10369E00E9FF600057F7EAFF020EEE24006E000EFF
:1036AE00EE20016E600053F7E1FF600057F7E2FF76
:1036BE00600003F0E6FF600007F0E6FF800EEE19F3
:1036CE00006E800E005C08E1000EED5D05E1000E5F
:1036DE00EC5D02E1000EEB5D18E2030EE313000E4B
:1036EE00E413006A016A026A036AEB51005EEC5150
:1036FE00015AED51025AEE51035A00C0EBF101C0CE
:10370E00ECF102C0EDF103C0EEF16CD0E3A937D0BD
:10371E00600053F7E9FF600057F7EAFF6F00B8FF4C
:10372E0000F06F00B8FF01F0600003F0E9FF6000E9
:10373E0007F0EAFF6F00B8FFEBF16F00B8FFECF196
:10374E006F00B8FFEDF16F00B8FFEEF1600053F7B8
:10375E00E9FF600057F7EAFF040EEE24006E000E3C
:10376E00EE20016E600053F7E1FF600057F7E2FFB5
:10377E00600003F0E6FF600007F0E6FF33D0600064
:10378E0053F7E9FF600057F7EAFF6F00B8FF00F04C
:10379E006F00B8FF01F0600003F0E9FF600007F072
:1037AE00EAFF6F00B8FFEBF16F00B8FFECF1000E0F
:1037BE00ED6FEE6F600053F7E9FF600057F7EAFF19
:1037CE00020EEE24006E000EEE20016E600053F726
:1037DE00E1FF600057F7E2FF600003F0E6FF6000D4
:1037EE0007F0E6FF000EDF1902E1000EDE190FE111
:1037FE00000E006EEE1908E10050ED1905E10050C3
:10380E00EC1902E1EB51000A02E1DE4BDF2BC00E98
:10381E00E315006E00C005F0BAD0010EE06FE05166
:10382E000A0A38E0E0C100F0000E016E026E036E6F
:10383E00003600900136023603360036009001360F
:10384E0002360336410E0024F66E500E0120F76E3E
:10385E00000E0220F86E09006F00D4FF01F009007F
:10386E006F00D4FF02F009006F00D4FF03F00900CF
:10387E006F00D4FF04F00450EE5D08E10350ED5DDF
:10388E0005E10250EC5D02E10150EB5D01E202D078
:10389E00E02BC5D78BD0010EE06FE051080A38E05F
:1038AE00E0C100F0000E016E026E036E0036009055
:1038BE0001360236033600360090013602360336E4
:1038CE000D0E0024F66E510E0120F76E000E022032
:1038DE00F86E09006F00D4FF01F009006F00D4FFED
:1038EE0002F009006F00D4FF03F009006F00D4FF4F
:1038FE0004F00450EE5D08E10350ED5D05E1025069
:10390E00EC5D02E10150EB5D01E202D0E02BC5D788
:10391E004DD0010EE06FE0510C0A38E0E0C100F02E
:10392E00000E016E026E036E0036009001360236F6
:10393E00033600360090013602360336E60E0024BA
:10394E00F66E4F0E0120F76E000E0220F86E090083
:10395E006F00D4FF01F009006F00D4FF02F00900E0
:10396E006F00D4FF03F009006F00D4FF04F0045081
:10397E00EE5D08E10350ED5D05E10250EC5D02E104
:10398E000150EB5D01E202D0E02BC5D70FD0055000
:10399E00000AD8B442D70550C00AD8B43ED7055055
:1039AE00800AD8B478D70550400AB3E0800E006E76
:1039BE00800EDF19005C02E1DE51E05D03E2DEC144
:1039CE00E0F10DD0800EDF19006E800E005C02E17A
:1039DE00E051DE5D04E2E0C1DEF1000EDF6FE15189
:1039EE00E2110EE0030EE315006EE4C101F0000ECD
:1039FE0001160050011004E0010EE15F000EE25BC3
:103A0E00800EDF19006E800EE219005C02E1E151BA
:103A1E00DE5D05E2DE51E15FDF51E25B02D0E16B7C
:103A2E00E26BC40EE315016EE451080B026E0250F8
:103A3E00080A02E1400E011808E1E151E21104E02A
:103A4E00010EE15F000EE25B1CD0C00EE315016EAD
:103A5E00E451080B026E0250080A02E1800E0118B2
:103A6E0010E1800E006E800EE219005C02E1E15161
:103A7E00020805E2020EE15F000EE25B02D0E16B8E
:103A8E00E26BE3A569D0E3A315D0E3A103D02D0E1D
:103A9E00DA6F02D02B0EDA6F60003FF7E1FF6000A5
:103AAE0043F7E2FF60006BF7E6FFCF4BD02BEF4BF7
:103ABE00F02B3BD0E3A10DD060003FF7E1FF60009B
:103ACE0043F7E2FF200EE66ECF4BD02BEF4BF02BE1
:103ADE002CD0C00EE315016EE451080B026E02509D
:103AEE00080A02E1800E011820E160003FF7E1FFB5
:103AFE00600043F7E2FF300EE66ECF4BD02BEF4B5C
:103B0E00F02BE3AB03D0580EDB6F02D0780EDB6FD9
:103B1E0060003FF7E1FF600043F7E2FF60006FF7E0
:103B2E00E6FFCF4BD02BEF4BF02BE151E21113E020
:103B3E0060003FF7E1FF600043F7E2FF300EE66EF4
:103B4E00CF4BD02BEF4BF02B010EE15F000EE25B63
:103B5E00E151E211EDE182D0E151E21115E0E3B75E
:103B6E0013D060003FF7E1FF600043F7E2FF200E45
:103B7E00E66ECF4BD02BEF4BF02B010EE15F000E1C
:103B8E00E25BE151E211EDE1E3A315D0E3A103D035
:103B9E002D0EDC6F02D02B0EDC6F60003FF7E1FFC5
:103BAE00600043F7E2FF600073F7E6FFCF4BD02BC8
:103BBE00EF4BF02B0ED0E3A10CD060003FF7E1FFEE
:103BCE00600043F7E2FF200EE66ECF4BD02BEF4B9B
:103BDE00F02BC00EE315016EE451080B026E02507D
:103BEE00080A02E1400E01180DE160003FF7E1FF07
:103BFE00600043F7E2FF300EE66ECF4BD02BEF4B5B
:103C0E00F02B2CD0C00EE315016EE451080B026EA2
:103C1E000250080A02E1800E011820E160003FF711
:103C2E00E1FF600043F7E2FF300EE66ECF4BD02B84
:103C3E00EF4BF02BE3AB03D0580EDD6F02D0780EB6
:103C4E00DD6F60003FF7E1FF600043F7E2FF6000C9
:103C5E0077F7E6FFCF4BD02BEF4BF02B800E006E9D
:103C6E00800EDF19005C02E1DE51E05D0DE26000C6
:103C7E003FF7E1FF600043F7E2FF300EE66ECF4BF9
:103C8E00D02BEF4BF02BEAD7DEC100F0DFC101F0F5
:103C9E00010EDE5F000EDF5B00500110D8B43FD185
:103CAE00C00EE315006E00C0F1F11CD1DEC100F0B4
:103CBE00DFC101F0000EDFBFFF0E026E036E003695
:103CCE000090013602360336003600900136023679
:103CDE000336410E0024F66E500E0120F76E000ED4
:103CEE000220F86E09006F00D4FF04F009006F0087
:103CFE00D4FF05F009006F00D4FF06F009006F0035
:103D0E00D4FF07F0EBC100F0ECC101F0EDC102F001
:103D1E00EEC103F028EC0CF00A0E046E000E056ED8
:103D2E00066E076E28EC0CF008C000F009C001F01A
:103D3E000AC002F00BC003F0300E0024E06FE1D099
:103D4E00E3AB4AD0DEC100F0DFC101F0000EDFBFF1
:103D5E00FF0E026E036E00360090013602360336F9
:103D6E00003600900136023603360D0E0024F66E34
:103D7E00510E0120F76E000E0220F86E09006F0042
:103D8E00D4FF04F009006F00D4FF05F009006F00A6
:103D9E00D4FF06F009006F00D4FF07F0EBC100F06E
:103DAE00ECC101F0EDC102F0EEC103F028EC0CF015
:103DBE000F0E0016000E0116021603166A0E0024D0
:103DCE00F66E520E0120F76E000E0220F86E0900FC
:103DDE006F00D4FFE0F149D0DEC100F0DFC101F089
:103DEE00000EDFBFFF0E026E036E0036009001362E
:103DFE0002360336003600900136023603360D0EBB
:103E0E000024F66E510E0120F76E000E0220F86EA1
:103E1E0009006F00D4FF04F009006F00D4FF05F015
:103E2E0009006F00D4FF06F009006F00D4FF07F001
:103E3E00EBC100F0ECC101F0EDC102F0EEC103F0F8
:103E4E0028EC0CF00F0E0016000E011602160316CB
:103E5E00590E0024F66E520E0120F76E000E02204F
:103E6E00F86E09006F00D4FFE0F14BD0DEC100F018
:103E7E00DFC101F0000EDFBFFF0E026E036E0036D3
:103E8E0000900136023603360036009001360236B7
:103E9E000336E60E0024F66E4F0E0120F76E000E6E
:103EAE000220F86E09006F00D4FF04F009006F00C5
:103EBE00D4FF05F009006F00D4FF06F009006F0073
:103ECE00D4FF07F0EBC100F0ECC101F0EDC102F040
:103EDE00EEC103F028EC0CF0070E0014E06F300E6C
:103EEE00E0270FD0F151000AD8B4E0D6F151C00A44
:103EFE00D8B4DCD6F151800AD8B422D7F151400A99
:103F0E00B5E060003FF7E1FF600043F7E2FF6000BD
:103F1E0083F7E6FFCF4BD02BEF4BF02BB5D6E3A7B5
:103F2E001CD0800E006E800EE219005C02E1E151A1
:103F3E00000813E260003FF7E1FF600043F7E2FF85
:103F4E00200EE66ECF4BD02BEF4BF02B010EE15F28
:103F5E00000EE25BE151E211EDE13CEF0EF0EFC13C
:083F6E0000F0F0C101F01200A7
:103F76000101D26B60003FF7E9FF600043F7EAFFFB
:103F86006F00B8FFD1F1D151000A10E0D1C1F7F1AD
:103F96007FEC09F00101D22BD251CF25E96E000E3C
:0E3FA600D021EA6E6F00B8FFD1F1EDD7120006
:0C3FB4006F00A0F701F001C000F0120047
:103FC00060003FF7F6FF600043F7F7FF600047F738
:103FD000F8FF09006F00D4FF00F0005216E0600007
:103FE0003FF7F6FF600043F7F7FF600047F7F8FF81
:103FF00009006F00D4FFFCF18DEC01F0010E01010E
:0C400000CF27000ED023D123DBD7120005
:10400C00086A096A100E0C6E013408360936045021
:10401C00085E0550D8A0053C095ED8B007D0045006
:10402C0008260550D8B0053C0926D8900036013634
:06403C000C2EEAD7120071
:0E404200550E3A01BF6FAA0EBF6FBF8112006C
:0E405000550E3A01BF6FAA0EBF6FBF9112004E
:10405E000101CF510308D8A0CF6BD0510308D8A0CF
:10406E00D06BF00E3D01F2170101CF513D01F2135D
:10407E00300EF213D0C100F00036009000360090E2
:10408E0000360090003600900050F413F38F1200AB
:10409E00CFC1B2F1D0C1B3F1D1C1B4F1D2C1B5F13A
:1040AE00D3C1B6F1D4C1B7F1D5C1B8F1D6C1B9F10A
:1040BE00D7C1BEF1D8C1BFF1D9C1C0F1DAC1C1F1CA
:1040CE00DBC1BAF1DCC1BBF1DDC1BCF1DEC1BDF1BA
:0240DE001200CE
:0C40E000C2C1CFF1C3C1D0F146DF120015
:1040EC00C70E0101CD6F010ECE6FC2C1CFF1C3C19E
:1040FC00D0F1C4C1D1F1C5C1D2F1C6C1D3F1CD0E3D
:10410C00D46F010ED56F37EC0EF000C0CBF101C0AF
:10411C00CCF10050C225E16E0150C321E26EE66A7B
:0A412C00CBC100F0CCC101F012007D
:104136000101C86BC96B000EC95D02E10A0EC85DBC
:104146000BE2C851C625E16EC951C721E26E200EA9
:10415600E66EC84BC92BEFD7C851C625E16EC951CB
:10416600C721E26EE66A010EC85F000EC95BC85140
:10417600C625CA6FC951C721CB6F0A0E046E000E41
:10418600056E066E076EC2C100F0C3C101F0C4C160
:1041960002F0C5C103F028EC0CF008C000F009C01D
:1041A60001F00AC002F00BC003F0300E00266000DA
:1041B6002BF7E1FF60002FF7E2FF600003F0E6FF58
:1041C6000A0E046E000E056E066E076EC2C100F082
:1041D600C3C101F0C4C102F0C5C103F028EC0CF064
:1041E60000C0C2F101C0C3F102C0C4F103C0C5F1F1
:1041F600000E046E031808E10450021805E104508D
:10420600011802E10050000A01E105D0010EC85F65
:08421600000EC95BACD71200D9
:04421E00CADE1200E2
:10422200310EB26E3C0EB16EB00EB06EC2C11DF157
:10423200C3C11EF13D6A3E6AB2803901A4919481E4
:02424200120068
:10424400B28AB288B280B282320EB26EB36A010E02
:10425400B56E3C0EB16EB00EB06E3901A49184817E
:1042640001011D6B1E6B3D6A3E6AB2903901949147
:02427400120036
:10427600FF0E0101CF6FFF0ED06F000ED16F000E43
:10428600D26F320ED36F030ED46FFC0ED56F010EB4
:10429600D66FFF0ED76FFF0ED86F000ED96F000EC8
:1042A600DA6FFF0EDB6FFF0EDC6F000EDD6F000EA8
:0C42B600DE6FF2DECF6BD06BCFDE1200AB
:1042C20009006F00D7FFE6FF0006FAE10106F8E1F8
:0242D2001200D8
:1042D400CA6A020E3A01406F830EC26EC294C29A39
:1042E400C298BA8ABA88BA84506BCB6AFF0EC36E7E
:1042F400FF0E516FC382C296BA963E01BC6BB86B77
:10430400FF0ECC6E800EC46E3A01606B9FDE130EFE
:10431400166F156B170EE56F92DEC49A618B61817F
:0E43240061836185629B6295629362911200D3
:10433200EF0E0101CF6F4E0ED06F000ED16F3FDE38
:104342003F01219521932181126B136B146B156B25
:10435200166B176B1E991E971E951E931E911E8F2C
:104362001E9B1F9F1F9D3901A19D919DA19B919B0A
:10437200FF0E3F011D6FFF0E1C6FFF0E1B6F1F977D
:104382001F951F931F911F9D250E0001C96F010EDE
:0E439200CA6F0101256B266B276B286B12008A
:1043A0000101C66B050EC65D0AE2C651C425E16E69
:1043B000000EC521E26E200EE66EC62BF3D7C65165
:1043C000C425E16E000EC521E26EE66AC607C6513D
:1043D000C425C76F000EC521C86F0A0E046E000EFB
:1043E000056EC2C100F0C3C101F010DE08C000F0CC
:1043F00009C001F0300E002660001FF7E1FF6000E9
:1044000023F7E2FF600003F0E6FF0A0E046E000EE1
:10441000056EC2C100F0C3C101F0F8DD00C0C2F1F9
:1044200001C0C3F1000E011802E1000E001801E105
:0844300002D0C607CCD7120030
:104438000D0E0101FC6F8DEC01F00A0E0101FC6FFD
:064448008DEC01F01200F2
:1044880000C01BF001C01AF03901A3A76ED093A792
:104498006CD06F00A0F7B1F13D01F9AB0FD0F99BDB
:1044A800010E01012B25006E000E2C21016E00C0AB
:1044B8002BF101C02CF16F00A0F7B1F13D01F9A774
:1044C8000ED0010E01012B25006E000E2C21016E6D
:1044D80000C02BF101C02CF19EDE00C0B1F101013A
:1044E800000E006E2A51005C02E129513E0817E2D5
:1044F80039019397010E01012D6F000E2E6F310EB9
:104508002925E16E010E2A21E26E6F0087FFE1FF87
:104518006F008BFFE2FFE66A3901949126D0010112
:104528002D6B2E6B310E2925E16E010E2A21E26ECC
:104538006F0087FFE1FF6F008BFFE2FF6000C7F6A7
:10454800E6FF010E2F25006E000E3021016E00C01F
:104558002FF101C030F1010E2925006E000E2A212D
:10456800016E00C029F101C02AF11BC000F01AC079
:0445780001F011003D
:10457C0052EC29F0600E3901D96F080EDF6F6E0016
:10458C0070F73FF0400E0101236F000E246F1F6B7C
:10459C00206B216B226B98DE290E0B6E960E0C6E27
:1045AC007F0E0D6E0D2EFED70C2EFCD70B2EFAD7D0
:1045BC00BA9801011B6B1C6B000E1C5D02E17F0E97
:1045CC001B5D10E2490E1B25E16E000E1C21E26EF4
:1045DC006F0087FFE1FF6F008BFFE2FFE66A1B4B6A
:1045EC001C2BEAD7490E476E000E486E400E3D015B
:1045FC00F56F030EF66FF28F38DEA30E0B6E570EAF
:10460C000C6E020E0D6E0D2EFED70C2EFCD70B2E43
:10461C00FAD7000039015B9109DF490E476E000E95
:10462C00486E1D0E0101CF6F520ED06F000ED16F70
:10463C00C1DC01011B6B1C6B000E1C5D02E1060E44
:10464C001B5D24E2030E006E000E016E1BC104F014
:10465C001CC105F048EC06F01C0E0024E96E000E9F
:10466C000120EA6E6F00A7FFE9FF6F00ABFFEAFFC6
:10467C006F00B8FFCFF16F00B8FFD0F16F00B8FF3B
:10468C00D1F198DC01011B4B1C2BD6D78A0ECF6FB6
:10469C00510ED06F000ED16F8DDC23C1C2F124C13D
:1046AC00C3F1CB0E0101C46F000EC56F73DECB0ED0
:1046BC00C26F000EC36F0EDDB9DED28E8B0E010100
:1046CC00CF6F500ED06F000ED16F74DCB5DD440E81
:1046DC003D01EA6FABDE500E0101C26F000EC36FDD
:1046EC009ADD000E3E1802E1000E3D1801E1F9D7EB
:1046FC00460E3D01EA6F9ADE99DE300E0101CF6F56
:10470C004F0ED06F000ED16F55DC650E0101CF6FCF
:10471C004E0ED06F000ED16F4DDC7B0E0101CF6FB2
:10472C00520ED06F000ED16F45DCFDDD250E000161
:10473C00C96F010ECA6F690E0101CF6F500ED06F99
:10474C00000ED16F37DC0101256B266B276B286BB4
:10475C003F01208B1F8FD00E0C6EC90E0D6E0D2ECF
:10476C00FED70C2EFCD7000000001F9F490E476E91
:10477C00000E486E600027F3E1FF60002BF3E2FFB0
:10478C006F004BFCE6FF010E0001C925E16E000E27
:10479C00CA21E26E6F0087FFE1FF6F008BFFE2FF23
:1047AC006F004FFCE6FF020EC925E16E000ECA2118
:1047BC00E26E6F0087FFE1FF6F008BFFE2FF6F007F
:1047CC0053FCE6FF030EC925E16E000ECA21E26E12
:1047DC006F0087FFE1FF6F008BFFE2FFE66AEE0ED2
:1047EC000101CF6F510ED06F000ED16FE0EC1FF0B6
:1047FC0001012851000808E12751000805E1265164
:10480C00000802E12551030806E2040E255F000EA4
:10481C00265B275B285B25C1C2F126C1C3F127C1EA
:10482C00C4F128C1C5F1CB0EC66F000EC76F7DDC7D
:10483C00CB0EC26F000EC36F4DDC2851000808E18F
:10484C002751000805E12651000802E125513F08D7
:10485C001FE2060E006E005007E028332733263384
:10486C002533289FFF0FF8D747C0C2F148C0C3F1CA
:10487C006B0EC46F510EC56F000EC66F25C1C7F10C
:10488C0026C1C8F127C1C9F128C1CAF129DC30D031
:10489C0025C100F026C101F027C102F028C103F0A8
:1048AC00C2EC05F0000E046E000E056E000E066ED6
:1048BC00790E076E47EC04F000C01FF101C020F127
:1048CC0002C021F103C022F147C0C2F148C0C3F1BC
:1048DC00CD0EC46F500EC56F000EC66F1FC1C7F151
:1048EC0020C1C8F121C1C9F122C1CAF176EC20F076
:1048FC0047C0C2F148C0C3F170EC20F097DD060E42
:10490C000101CF6F520ED06F000ED16FE0EC1FF093
:10491C003F011F971F951F931F911F9D0101256B31
:10492C00266B276B286B3F01208BBA9820B102D0E5
:10493C00BA9A01D0BA8A1F8F150E0C6EC60E0D6E68
:10494C000D2EFED70C2EFCD700001F9F20B102D0DD
:10495C00BA9A01D0BA8ABA88600027F3E1FF6000E6
:10496C002BF3E2FF6F004BFCE6FF010E0001C925A3
:10497C00E16E000ECA21E26E6F0087FFE1FF6F004F
:10498C008BFFE2FF6F004FFCE6FF020EC925E16EC4
:10499C00000ECA21E26E6F0087FFE1FF6F008BFFF4
:1049AC00E2FF6F0053FCE6FF030EC925E16E000E1B
:1049BC00CA21E26E6F0087FFE1FF6F008BFFE2FF01
:1049CC00E66AD60E0101CF6F510ED06F000ED16F7B
:1049DC00E0EC1FF001012851000808E12751000804
:1049EC0005E12651000802E12551030806E2040EF8
:1049FC00255F000E265B275B285B25C1C2F126C113
:104A0C00C3F127C1C4F128C1C5F1CB0EC66F000E8E
:104A1C00C76F9BEC20F0CB0EC26F000EC36F70EC17
:104A2C0020F02851000808E12751000805E1265123
:104A3C00000802E125513F0820E2060E006E0050EE
:104A4C0007E02833273326332533289FFF0FF8D769
:104A5C0047C0C2F148C0C3F12D0EC46F510EC56FD3
:104A6C00000EC66F25C1C7F126C1C8F127C1C9F117
:104A7C0028C1CAF176EC20F030D025C100F026C157
:104A8C0001F027C102F028C103F0C2EC05F0000EC2
:104A9C00046E000E056E000E066E790E076E47EC66
:104AAC0004F000C01FF101C020F102C021F103C0CD
:104ABC0022F147C0C2F148C0C3F1AD0EC46F500E15
:104ACC00C56F000EC66F1FC1C7F120C1C8F121C14F
:104ADC00C9F122C1CAF176EC20F047C0C2F148C03E
:104AEC00C3F170EC20F0A2DCA50E0101CF6F510ECA
:104AFC00D06F000ED16FE0EC1FF03F011F971F9598
:104B0C001F931F911F9D0101256B266B276B286B33
:104B1C003F01208BBA9820B102D0BA9A01D0BA8A40
:104B2C001F8F0000000000000000000000000000CB
:104B3C0000001F9F20B102D0BA9A01D0BA8ABA885D
:104B4C00600027F3E1FF60002BF3E2FF6F004BFCEA
:104B5C00E6FF010E0001C925E16E000ECA21E26ECE
:104B6C006F0087FFE1FF6F008BFFE2FF6F004FFCD0
:104B7C00E6FF020EC925E16E000ECA21E26E6F003F
:104B8C0087FFE1FF6F008BFFE2FF6F0053FCE6FF36
:104B9C00030EC925E16E000ECA21E26E6F0087FF7D
:104BAC00E1FF6F008BFFE2FFE66ABE0E0101CF6FE3
:104BBC00510ED06F000ED16FE0EC1FF001012851A7
:104BCC00000808E12751000805E12651000802E120
:104BDC002551030806E2040E255F000E265B275BB9
:104BEC00285B25C1C2F126C1C3F127C1C4F128C17C
:104BFC00C5F1CB0EC66F000EC76F9BEC20F0CB0E31
:104C0C00C26F000EC36F70EC20F02851000808E151
:104C1C002751000805E12651000802E125513F0803
:104C2C0020E2060E006E005007E0283327332633AF
:104C3C002533289FFF0FF8D747C0C2F148C0C3F1F6
:104C4C004C0EC46F510EC56F000EC66F25C1C7F157
:104C5C0026C1C8F127C1C9F128C1CAF176EC20F0F0
:104C6C0030D025C100F026C101F027C102F028C1C7
:104C7C0003F0C2EC05F0000E046E000E056E000E83
:104C8C00066E790E076E47EC04F000C01FF101C0F0
:104C9C0020F102C021F103C022F147C0C2F148C08B
:104CAC00C3F1ED0EC46F500EC56F000EC66F1FC161
:104CBC00C7F120C1C8F121C1C9F122C1CAF176ECFA
:104CCC0020F047C0C2F148C0C3F170EC20F01CECDE
:104CDC0022F0320E0101CF6F520ED06F000ED16F49
:104CEC00E0EC1FF0020E0A6E960E0B6ED80E0C6ED8
:104CFC00080E0D6E0D2EFED70C2EFCD70B2EFAD7F0
:104D0C000A2EF8D700008A0E0101CF6F520ED06F19
:0C4D1C00000ED16FE0EC1FF0FF00FFD78D
:104D5C0000C019F001C018F0390194A120D0A4A111
:104D6C001ED0010E01011D5D006E000E1E59016E5C
:104D7C0000C01DF101C01EF1000E1E5D02E1010E0E
:104D8C001D5D07E239019491B290010E3D6E000E4B
:104D9C003E6E39013C0EB16EB00EB06EA49119C0CE
:084DAC0000F018C001F0110035
:1052A40010EE1CF02B0E006E010E016E160EF66E43
:0E52B400500EF76E000EF86E61EC21F0120045
:10444E002050726F6A6574203A31384632374B34D9
:10445E00325F54657374735F534D54315F6368728A
:10446E006F6E6F6D657472655F323032325F3038E9
:09447E002E6D637070690D0A00D7
:104D28000000007FCDCC4C7B0AD723786F12037527
:104D380017B75171ACC5276EBD37066B95BF56675F
:104D480077CC2B645F700961FFE65B5D08E53C3C4E
:044D58006042221B78
:104DB40020436F6E66696720626974203A20205030
:104DC40031384632374B34325F466F73635F496E16
:104DD4007465726E655F4956545F696E746572726C
:104DE400757074735F313678345F504C4C5F363471
:104DF4004D487A2E6366677363682020464F534399
:0C4E04003A36342E30204D487A0D0A005A
:104E1000204469726563746F7279203A433A5C5F2B
:104E20004D696B726F435C5F4D657350726F6A655D
:104E300074735F4D696B726F435C5F313846323714
:104E40004B34325F54657374735F534D54315F63F9
:104E500068726F6E6F6D657472655F323032325F8B
:054E600030380D0A00CE
:104E6500205265736F6C7574696F6E20636F6D701A
:104E750074657572202B2D203136206E616E6F534F
:104E850065632028647572E965206D6178696D61D7
:104E9500206D6573757261626C65203D2032363216
:064EA5006D53290D0A0007
:104EAB0020536F75726365203A2050494331384661
:104EBB0032374B34325F746573745F534D54315FCB
:104ECB004368726F6E6F6D657472655F55415254B6
:104EDB005F4956545F5F323032325F303832352E95
:044EEB00630D0A0049
:104EEF00205465737420534D5420636F6D70746537
:104EFF0075722032342062697473202872E97375D9
:104F0F006DE92064657320726567697374726573E8
:104F1F0020656E20706167652033363429200D0AB5
:014F2F000081
:104F3000205465737420636F6D70746575722032D0
:104F400034206269747320534D543120737572207C
:104F5000464F53433D36344D487A20656E206D6F81
:104F60006465206368726F6E6F6D657472650D0A9B
:014F70000040
:104F710020546573742050494331384632374B34DD
:104F8100322049565420657420636F6D70746575C5
:104F910072203234206269747320534D543120657C
:104FA1006E206368726F6E6F6D65747265200D0A95
:014FB10000FF
:104FB2000000007F000020820000488500007A88FF
:104FC20000401C8C0050438F0024749280961896E7
:104FD20020BC3E99286B6E9CF90215A0EC782DC17D
:044FE200CAF249E2E4
:104FE6000100000008000000400000000002000070
:104FF60000100000008000000000040000002000F7
:105006000000000100000008000000400000000051
:10501600104E004652004E4400714F00B44D00AB96
:105026004E009C52009752009E5200A05200A2527F
:015036000079
:02503700000077
:015039000076
:07503A00286E756C6C290063
:10504100010000000A00000064000000E803000005
:1050510010270000A086010040420F0080969800B2
:0850610000E1F50500CA9A3BCD
:1050690020537461727420534D543120666F72203D
:10507900746573742064656C61792031306D530DEA
:025089000A001B
:10508B0020546573742054696D6572312038307803
:10509B0032356D7320736F69742032736563200D25
:0250AB000A00F9
:1050AD00202C6574202876696120737072696E7486
:1050BD006629202D3E2025332E3366207553200082
:1050CD00202C6574202876696120737072696E7466
:1050DD006629202D3E2025332E3366207553200062
:1050ED00202C6574202876696120737072696E7446
:1050FD006629202D3E2025332E3366207553200042
:10510D000100000010000000000100000010000070
:10511D000000010000001000000000010000001060
:10512D00202C206574202876696120737072696E59
:0F513D00746629202D3E20256C752075532000A7
:10514C00202C206574202876696120737072696E3A
:0F515C00746629202D3E20256C75207553200088
:10516B00202C206574202876696120737072696E1B
:0F517B00746629202D3E20256C75207553200069
:10518A002020436C6F636B20696E697469616C657A
:0B519A0020696E204D487A203D200067
:1051A500205465737420534D543120737572203823
:0951B500204E4F5020200D0A008D
:1051BE002053746F702E0D0A20534D543120746994
:0851CE00637320202D3E200038
:1051D6002053746F702E0D0A20534D54312074697C
:0851E600637320202D3E200020
:1051EE002053746F702E0D0A20534D543120746964
:0851FE00637320202D3E200008
:10520600205465737420534D5431207375722031C8
:075216006D5320200D0A007A
:10521D000D0A2050726573656E746174696F6E202E
:05522D003A200D0A000B
:1052320046696E2064652074657374202E2E2E21BB
:045242000D0A200031
:10524600204D696B726F432070726F20372E363097
:035256000D0A003E
:1052590030313233343536373839616263646566E3
:015269000044
:10526A003031323334353637383941424344454692
:01527A000033
:0F527B0020496E69742020534D5431200D0A00D4
:0D528A00205265626F6F7420210D0A200014
:0552970020200D0A00BB
:02529C002000F0
:02529E002000EE
:0252A0002000EC
:0252A2002000EA
:020000040030CA
:0A00000024292DA70B3F9F0F0100DC
:00000001FF
